:020000040000FA
:06000000A7EF23F012003F
:06140000A7EF23F012002B
:021408001200D0
:021418001200C0
:06142A0002007047000003
:10143000C10000000B0000006C470000D600000057
:0414400004000000A4
:0C14440072EC11F0030A01E1E9D3010A87
:1014500001E1FCD1030A0CE00001725102E127EF27
:1014600010F00001785102E127EF10F012EF10F0B8
:10147000C60EE66E010EE66E0D0EE66E900EE66E80
:1014800000EC21F0E552E552E552E552E66A010E24
:10149000E66E2C0EE66E22EC22F0E552E552E552A5
:1014A000C6C176F00001776BC6C177F0766B000E8F
:1014B0007617FF0E7717E00E0101C715000176259C
:1014C000766F000E772176C000F0016E050ED89081
:1014D00001320032E804FBE100C076F001C077F091
:1014E0000F0E0001001819E1030E771916E1580ECE
:1014F0000101CF5D02E0000E01D0010E006E180E5A
:10150000CF5D02E0000E01D0010E001003E00001EB
:10151000836B03D00001010E836F0F0E000176195B
:1015200019E1030E771916E1480E0101CF5D02E0C3
:10153000000E01D0010E006E080ECF5D02E0000E1D
:1015400001D0010E001003E00001846B03D0000104
:10155000010E846F5F0E000176190DE1030E7719FD
:101560000AE1040E0101D25D06E161C0AFF062C084
:10157000B0F063C0B1F0AF0EE96E000EEA6EEE504F
:101580000001615D026EEE506259036EEE506359C8
:10159000046ED880640E0254000E0354000E0454EE
:1015A00002E2000E01D0010E016E400E0101CD15C8
:1015B000400802E0000E01D0010E006E7F0E000117
:1015C000761902E1010E771902E0000E01D0010E3A
:1015D0000014011403E00001010E796F400E0101B7
:1015E000CD15400802E1000E01D0010E006E7F0E05
:1015F0000001761902E1010E771902E0000E01D018
:10160000010E001402E00001796BAF0EE96E000ECE
:10161000EA6EEE500001615D006EEE506259016E9F
:10162000EE506359026ED880640E0054000E0154CF
:10163000000E025402E20001796B7F0E0001761960
:1016400016E1010E771913E1060E0101CE15060809
:1016500004E10001010E7A6F0AD000017A0506E16B
:1016600061C07EF062C07FF063C080F07A6B0001E1
:101670007A5102E0F7EF0FF07F0E000176190CE1CE
:10168000010E771909E10001720506E10101060E5C
:10169000CE6F0001010E946F5F0E0001761901E01C
:1016A0007ED0030E771901E07AD07B0EE96E000E32
:1016B000EA6EEE500001615D006EEE506259016EFF
:1016C000EE506359026E040E005C000E0158000ECD
:1016D000025865E3020E0101D25D28E16C0EE96E4D
:1016E000000EEA6EEE500001615D006EEE50625930
:1016F000016EEE506359026EA00E005C000E0158A0
:10170000000E025813E2899289900001726B000169
:10171000A40E6C6F6D6B6E6B0001696F6A6B6B6B07
:1017200061C07BF062C07CF063C07DF00101CD053B
:1017300002E0000E01D0010E006ED20502E0000EA4
:1017400001D0010E00102BE0690EE96E000EEA6E6A
:10175000EE500001615D006EEE506259016EEE5078
:101760006359026EA00E005C000E0158000E025874
:1017700016E20001905113E1899289900001726B89
:101780000001A40E6C6F6D6B6E6B0001696F6A6B6C
:101790006B6B61C07BF062C07CF063C07DF05F0E5C
:1017A0000001761902E0F7EF0FF0030E771902E05F
:1017B000F7EF0FF07B0EE96E000EEA6EEE500001BF
:1017C000615D006EEE506259016EEE506359026E1B
:1017D000040E005C000E0158000E025802E2F7EF02
:1017E0000FF0020E0101D25D05E10001010E646FF0
:1017F0000001656B0101D20505E10001010E656F75
:101800000001646B0101CD0505E10001010E656F6A
:101810000001646B0101CD0501E1E9D3110EE76E12
:10182000D219E8AE02D0E73402D0E750D25D01E22F
:10183000DED3150EE76ED219E8AE02D0D23503D052
:10184000E750D880D25501E2D2D3CDD3C60EE66E92
:10185000010EE66E0D0EE66E940EE66E00EC21F0C3
:10186000E552E552E552E552E66A020EE66E2C0EAE
:10187000E66E22EC22F0E552E552E552C6C176F062
:101880000001776BC6C177F0766B000E7617FF0EFE
:101890007717E00E0101C71500017625766F000E5F
:1018A000772176C000F0016E050ED890013200322B
:1018B000E804FBE100C076F001C077F00F0E0001F4
:1018C000001819E1030E771916E1580E0101CF5DDA
:1018D00002E0000E01D0010E006E180ECF5D02E096
:1018E000000E01D0010E001003E00001836B03D055
:1018F0000001010E836F0F0E0001761919E1030E2E
:10190000771916E1480E0101CF5D02E0000E01D00B
:10191000010E006E080ECF5D02E0000E01D0010E38
:10192000001003E00001846B03D00001010E846FFE
:101930005F0E000176190DE1030E77190AE1040E1E
:101940000101D25D06E161C0AFF062C0B0F063C0DA
:10195000B1F0AF0EE96E000EEA6EEE500001615D6F
:10196000026EEE506259036EEE506359046ED880D9
:10197000640E0254000E0354000E045402E2000EE2
:1019800001D0010E016E400E0101CD15400802E0AC
:10199000000E01D0010E006E7F0E0001761902E1EB
:1019A000010E771902E0000E01D0010E001401149F
:1019B00003E00001010E796F400E0101CD154008D2
:1019C00002E1000E01D0010E006E7F0E00017619BB
:1019D00002E1010E771902E0000E01D0010E0014A1
:1019E00002E00001796BAF0EE96E000EEA6EEE5078
:1019F0000001615D006EEE506259016EEE50635958
:101A0000026ED880640E0054000E0154000E025481
:101A100002E20001796B7F0E0001761916E1010EDA
:101A2000771913E1060E0101CE15060804E1000145
:101A3000010E7A6F0AD000017A0506E161C07EF0DE
:101A400062C07FF063C080F07A6B00017A5101E0E0
:101A5000CED27F0E000176190CE1010E771909E153
:101A60000001720506E10101060ECE6F0001010EB4
:101A7000946F5F0E0001761901E07ED0030E771996
:101A800001E07AD07B0EE96E000EEA6EEE500001A6
:101A9000615D006EEE506259016EEE506359026E48
:101AA000040E005C000E0158000E025865E3020EA1
:101AB0000101D25D28E16C0EE96E000EEA6EEE5077
:101AC0000001615D006EEE506259016EEE50635987
:101AD000026EA00E005C000E0158000E025813E2C8
:101AE000899289900001726B0001A40E6C6F6D6B7E
:101AF0006E6B0001696F6A6B6B6B61C07BF062C0DB
:101B00007CF063C07DF00101CD0502E0000E01D044
:101B1000010E006ED20502E0000E01D0010E001091
:101B20002BE0690EE96E000EEA6EEE500001615D79
:101B3000006EEE506259016EEE506359026EA00EB7
:101B4000005C000E0158000E025816E20001905190
:101B500013E1899289900001726B0001A40E6C6FF1
:101B60006D6B6E6B0001696F6A6B6B6B61C07BF0B4
:101B700062C07CF063C07DF05F0E0001761901E069
:101B800036D2030E771901E032D27B0EE96E000ED9
:101B9000EA6EEE500001615D006EEE506259016E1A
:101BA000EE506359026E040E005C000E0158000EE8
:101BB000025801E21CD2020E0101D25D05E10001D2
:101BC000010E646F0001656B0101D20505E10001A2
:101BD000010E656F0001646B0101CD0505E1000197
:101BE000010E656F0001646B0101CD0501E1FFD1BC
:101BF000110EE76ED219E8AE02D0E73402D0E750FA
:101C0000D25D01E2F4D1150EE76ED219E8AE02D032
:101C1000D23503D0E750D880D25501E2E8D1E3D1E4
:101C2000C60EE66E010EE66E0D0EE66E900EE66EC8
:101C300000EC21F0E552E552E552E552E66A010E6C
:101C4000E66E2C0EE66E22EC22F0E552E552E552ED
:101C5000C6C176F00001776BC6C177F0766B000ED7
:101C60007617FF0E7717E00E0101C71500017625E4
:101C7000766F000E772176C000F0016E050ED890C9
:101C800001320032E804FBE100C076F001C077F0D9
:101C90000F0E0001001819E1030E771916E1580E16
:101CA0000101CF5D02E0000E01D0010E006E180EA2
:101CB000CF5D02E0000E01D0010E001003E0000134
:101CC000836B03D00001010E836F0F0E00017619A4
:101CD00019E1030E771916E1480E0101CF5D02E00C
:101CE000000E01D0010E006E080ECF5D02E0000E66
:101CF00001D0010E001003E00001846B03D000014D
:101D0000010E846F5F0E000176190DE1030E771945
:101D10000AE1040E0101D25D06E161C0AFF062C0CC
:101D2000B0F063C0B1F0AF0EE96E000EEA6EEE5097
:101D30000001615D026EEE506259036EEE50635910
:101D4000046ED880640E0254000E0354000E045436
:101D500002E2000E01D0010E016E400E0101CD1510
:101D6000400802E0000E01D0010E006E7F0E00015F
:101D7000761902E1010E771902E0000E01D0010E82
:101D80000014011403E00001010E796F400E0101FF
:101D9000CD15400802E1000E01D0010E006E7F0E4D
:101DA0000001761902E1010E771902E0000E01D060
:101DB000010E001402E00001796BAF0EE96E000E17
:101DC000EA6EEE500001615D006EEE506259016EE8
:101DD000EE506359026ED880640E0054000E015418
:101DE000000E025402E20001796B7F0E00017619A9
:101DF00016E1010E771913E1060E0101CE15060852
:101E000004E10001010E7A6F0AD000017A0506E1B3
:101E100061C07EF062C07FF063C080F07A6B000129
:101E20007A5101E0E4D07F0E000176190CE1010E39
:101E3000771909E10001720506E10101060ECE6F76
:101E40000001010E946F5F0E0001761901E07ED053
:101E5000030E771901E07AD07B0EE96E000EEA6E70
:101E6000EE500001615D006EEE506259016EEE5061
:101E70006359026E040E005C000E0158000E0258F9
:101E800065E3020E0101D25D28E16C0EE96E000EE1
:101E9000EA6EEE500001615D006EEE506259016E17
:101EA000EE506359026EA00E005C000E0158000E49
:101EB000025813E2899289900001726B0001A40E0E
:101EC0006C6F6D6B6E6B0001696F6A6B6B6B61C0E1
:101ED0007BF062C07CF063C07DF00101CD0502E0C3
:101EE000000E01D0010E006ED20502E0000E01D0FE
:101EF000010E00102BE0690EE96E000EEA6EEE5046
:101F00000001615D006EEE506259016EEE50635942
:101F1000026EA00E005C000E0158000E025816E280
:101F20000001905113E1899289900001726B0001C8
:101F3000A40E6C6F6D6B6E6B0001696F6A6B6B6BDF
:101F400061C07BF062C07CF063C07DF05F0E000179
:101F500076194DE1030E77194AE17B0EE96E000E0A
:101F6000EA6EEE500001615D006EEE506259016E46
:101F7000EE506359026E040E005C000E0158000E14
:101F8000025835E3020E0101D25D05E10001010EA8
:101F9000646F0001656B0101D20505E10001010ECE
:101FA000656F0001646B0101CD0505E10001010EC3
:101FB000656F0001646B0101CD0519E0110EE76E3C
:101FC000D219E8AE02D0E73402D0E750D25D0FE379
:101FD000150EE76ED219E8AE02D0D23503D0E75025
:101FE000D880D25504E30001646B0001656BC60E16
:101FF000E66E010EE66E0D0EE66EE668F7EC1EF07C
:10200000E552E552E552E55261C073F062C074F0EA
:1020100063C075F0E66A2D0EE66E59EC20F0E552CD
:10202000E55215D0C60EE66E010EE66E0D0EE66E9A
:10203000E668F7EC1EF0E552E552E552E55261C064
:1020400073F062C074F063C075F00001786B1AD948
:10205000030A01E1F1D0010A01E1DDD0030A01E048
:102060001200A60EE66E010EE66E0D0EE66E900EE6
:10207000E66EBAEC1EF0E552E552E552E552E66A2C
:10208000010EE66E2C0EE66EDCEC1FF0E552E5521A
:10209000E552A6C176F00001776BA6C177F0766BAA
:1020A000000E7617FF0E7717E00E0101A71500014D
:1020B0007625766F000E772176C000F0016E050E52
:1020C000D89001320032E804FBE100C076F001C094
:1020D00077F000017A5131E1100E0101B2150001D3
:1020E000C16FDF0E0001761928E1030E771925E193
:1020F0000001720522E1100E0001C15D1EE16F0EAC
:10210000E96E000EEA6EEE500001615D006EEE5069
:102110006259016EEE506359026ED880100E005461
:10212000000E0154000E025408E261C06FF062C05C
:1021300070F063C071F089928990DF0E000176190A
:1021400001E092D0030E771901E08ED0B2C196F073
:10215000690EE96E000EEA6EEE500001615D006EE0
:10216000EE506259016EEE506359026EA00E005C93
:10217000000E0158000E02581CE20001965119E1B0
:10218000899289900001726B0001A40E6C6F6D6BD7
:102190006E6B0001696F6A6B6B6B61C07BF062C034
:1021A0007CF063C07DF00001946B0001AF6FB06BF9
:1021B000B16B6C0EE96E000EEA6EEE500001615DCF
:1021C000006EEE506259016EEE506359026EA00E21
:1021D000005C000E0158000E025846E20001960510
:1021E00043E1899289900001726B0001A40E6C6F2B
:1021F0006D6B6E6B0001696F6A6B6B6B61C07BF01E
:1022000062C07CF063C07DF00001946B0001AF6F91
:10221000B06BB16B29D0A60EE66E010EE66E0D0E08
:10222000E66E940EE66EBAEC1EF0E552E552E5520B
:10223000E552E66A020E10D0A60EE66E010EE66EBC
:102240000D0EE66E900EE66EBAEC1EF0E552E5520B
:10225000E552E552E66A010EE66E2C0EE66EDCEC07
:102260001FF0E552E552E552A60EE66E010EE66E4F
:102270000D0EE66EE6683DEC21F0E552E552E552C2
:10228000E5521200D9CFE6FFE1CFD9FFE6520101B6
:10229000FD93FD95A9EC1FF0DF6EDFA00CD00101CE
:1022A000FD51060BE8420109030BF36EF346F90EEC
:1022B000FD15F310FD6FDFA20CD00101FD51060BDF
:1022C000E8420209030BF36EF346F90EFD15F31015
:1022D000FD6F0101FD51060BE842E552E552E7CFE3
:1022E000D9FF1200D9CFE6FFE1CFD9FFE6520101B5
:1022F000FE93FE95EFEC21F0DF6EDFA00CD0010124
:10230000FE51060BE8420109030BF36EF346F90E8A
:10231000FE15F310FE6FDFA20CD00101FE51060B7B
:10232000E8420209030BF36EF346F90EFE15F310B3
:10233000FE6F0101FE51060BE842E552E552E7CF80
:10234000D9FF1200D9CFE6FFE1CFD9FFE652898449
:102350009294E66AE66A010EE66E02EC23F0E5521C
:10236000E552E552938A9398DF6ADFCF00F0400E82
:10237000E76E0018E8AE02D0E73402D0E750005C08
:1023800016E2DFCFE9FFEA6AE9BEEA68050EE92650
:10239000010EEA22EF6ADFCFE9FFEA6AE9BEEA68E6
:1023A000450EE926010EEA22EF6ADF2ADED7480E43
:1023B000D76EE40ED66ED596D584D592D580D59AB3
:1023C000D59C49D8E552E552E7CFD9FF1200D9CFC5
:1023D000E6FFE1CFD9FFE65289869296E66AE66A81
:1023E000010EE66ED7EC22F0E552E552E552DF6AC7
:1023F000DFCF00F0400EE76E0018E8AE02D0E73401
:1024000002D0E750005C16E2DFCFE9FFEA6AE9BEDE
:10241000EA68050EE926010EEA22EF6ADFCFE9FF3E
:10242000EA6AE9BEEA68450EE926010EEA22EF6A89
:10243000DF2ADED7480ED76EE40ED66ED596D58449
:10244000D592D580D59A0101FD9D3DD9E552E55241
:10245000E7CFD9FF1200D9CFE6FFE1CFD9FFE6528F
:10246000FCEC1DF0DF6ADF50006E016AD89001506D
:1024700004E6FA0E005C000E015802E2DF2AF3D7F0
:102480000001B38FB39DB39BB397B399B395B3C01A
:10249000E6FF0F0EE66E13EC1EF0E552E5520E0E4F
:1024A000E66E5DEC1EF0E552E00B800808E0B3C07C
:1024B000E6FF0F0EE66E13EC1EF0E552E552010149
:1024C000866B876B886B896B860EE66E010EE66EF7
:1024D000040EE66E200EE66E2EEC1EF0E552E5527E
:1024E000E552E552860EE66E010EE66E040EE66ECD
:1024F000240EE66E2EEC1EF0E552E552E552E55252
:10250000E66A010EE66E13EC1EF0E552E552E66A4D
:10251000050EE66E13EC1EF0E552E552080EE66E6F
:10252000090EE66E13EC1EF0E552E552080EE66E5B
:10253000110EE66E13EC1EF0E552E552080EE66E43
:10254000150EE66E13EC1EF0E552E552080EE66E2F
:10255000190EE66E13EC1EF0E552E5520101A30ED2
:10256000866F090E876F120E886F340E896F040E06
:102570008A6F8B6B010E8C6F020E8D6F030E8E6F48
:10258000040E8F6F050E906F060E916F070E926FFF
:10259000860EE66E010EE66E0D0EE66E400EE66EDF
:1025A000F7EC1EF0E552E552E552E5520101220E2C
:1025B000866F876B640E886F680E896F020E8A6F54
:1025C0008B6B110E8C6F220E8D6F330E8E6F440E3F
:1025D0008F6F550E906F660E916F770E926F860E0D
:1025E000E66E010EE66E0D0EE66E420EE66EF7EC3E
:1025F0001EF0E552E552E552E5520101AA0E866F42
:10260000030E876F330E886F896F080E8A6FAA0ECC
:102610008B6FBB0E8C6FCC0E8D6FDD0E8E6FEE0E42
:102620008F6F90690A0E916F0B0E926F860EE66E99
:10263000010EE66E0D0EE66E440EE66EF7EC1EF031
:10264000E552E552E552E5520001B68F070EE66EFF
:102650007CD9E5520001B39FB39DB39BB3C0E6FFA5
:102660000F0EE66E13EC1EF0E552E5520101856B8C
:102670000E0EE66E5DEC1EF0E552E00B08E0B3C016
:10268000E6FF0F0EE66E13EC1EF0E552E552000178
:10269000BA85BA91BA87BA93BAC0E6FF0C0EE66E55
:1026A00013EC1EF0E552E552E668300EE66E0C0EB5
:1026B000E66EDCEC1FF0E552E552E552E552E552DC
:1026C000E7CFD9FF1200D9CFE6FFE1CFD9FFE6521D
:1026D00042EC20F0DF6ADF50006E016AD8900150B2
:1026E00004E6FA0E005C000E015802E2DF2AF3D77E
:1026F0000001B38FB39DB39BB397B399B385B393E5
:10270000B391B3C0E6FF0F0EE66E59EC20F0E55230
:10271000E5520E0EE66EA3EC20F0E552E00B8008C9
:1027200008E0B3C0E6FF0F0EE66E59EC20F0E5526C
:10273000E5520101866B876B886B896B860EE66EAE
:10274000010EE66E040EE66E200EE66E74EC20F0CE
:10275000E552E552E552E552860EE66E010EE66E52
:10276000040EE66E240EE66E74EC20F0E552E5529F
:10277000E552E552BFC0E6FF600EE66E59EC20F070
:10278000E552E552E66A010EE66E59EC20F0E5529C
:10279000E552E66A050EE66E59EC20F0E552E55288
:1027A000080EE66E090EE66E59EC20F0E552E55291
:1027B000080EE66E110EE66E59EC20F0E552E55279
:1027C000080EE66E150EE66E59EC20F0E552E55265
:1027D000080EE66E190EE66E59EC20F0E552E55251
:1027E0000101A30E866F090E876F120E886F340EDB
:1027F000896F040E8A6F8B6B010E8C6F020E8D6FCA
:10280000030E8E6F040E8F6F050E906F060E916F84
:10281000070E926F860EE66E010EE66E0D0EE66EE8
:10282000400EE66E3DEC21F0E552E552E552E552F0
:102830000101220E866F876B640E886F680E896FA8
:10284000020E8A6F8B6B110E8C6F220E8D6F330E02
:102850008E6F440E8F6F550E906F660E916F770ED0
:10286000926F860EE66E010EE66E0D0EE66E420E5D
:10287000E66E3DEC21F0E552E552E552E5520101EC
:10288000AA0E866F030E876F330E886F896F080E4E
:102890008A6FAA0E8B6FBB0E8C6FCC0E8D6FDD0E08
:1028A0008E6FEE0E8F6F90690A0E916F0B0E926F06
:1028B000860EE66E010EE66E0D0EE66E440EE66EB8
:1028C0003DEC21F0E552E552E552E5520001B68FAC
:1028D000070EE66EC9D8E5520001B39FB39DB39BC6
:1028E000B3C0E6FF0F0EE66E59EC20F0E552E5525C
:1028F0000101856B0E0EE66EA3EC20F0E552E00BB5
:1029000008E0B3C0E6FF0F0EE66E59EC20F0E5528A
:10291000E5520001BA85BA91BA87BA93BAC0E6FF08
:102920000C0EE66E59EC20F0E552E552E66A300EE8
:10293000E66E0C0EE66E22EC22F0E552E552E55210
:10294000E552E552E7CFD9FF1200D9CFE6FFE1CF3C
:10295000D9FF040EE1260001B38FB39DB39BB3C032
:10296000E6FF0F0EE66E13EC1EF0E552E5520E0E7A
:10297000E66E5DEC1EF0E552E00B800808E0B3C0A7
:10298000E6FF0F0EE66E13EC1EF0E552E552000175
:10299000B46B0001B56B0001B66B0001B49FB49D30
:1029A0000001B595B583B591B59BB589B597000183
:1029B000B695B683B6910001B58FB58DFE0EDB508E
:1029C00015E0010A0EE0020A07E0040A13E1C00E56
:1029D0000001B415070F0DD0C00E0001B415030F90
:1029E00008D0C00E0001B415010F03D0C00E0001C5
:1029F000B415B46FB6C086F1B5C087F1B4C088F124
:102A0000860EE66E010EE66E030EE66E280EE66E8C
:102A10002EEC1EF0E552E552E552E5520001B39F5F
:102A2000B39DB39BB3C0E6FF0F0EE66E13EC1EF032
:102A3000E552E5520E0EE66E5DEC1EF0E552E00B3F
:102A4000800808E0B3C0E6FF0F0EE66E13EC1EF040
:102A5000E552E552040EE15C02E2E16AE552E16E04
:102A6000E552E7CFD9FF1200D9CFE6FFE1CFD9FF7A
:102A7000040EE1260001B38FB39DB39BB3C0E6FF04
:102A80000F0EE66E59EC20F0E552E5520E0EE66EA2
:102A9000A3EC20F0E552E00B800808E0B3C0E6FFAD
:102AA0000F0EE66E59EC20F0E552E5520001B46BD2
:102AB0000001B56B0001B66B0001B49FB49D00012D
:102AC000B595B583B591B59BB589B5970001B69518
:102AD000B683B6910001B58FB58DFE0EDB5015E0C3
:102AE000010A0EE0020A07E0040A13E1C00E000129
:102AF000B415070F0DD0C00E0001B415030F08D098
:102B0000C00E0001B415010F03D0C00E0001B415B2
:102B1000B46FB6C086F1B5C087F1B4C088F1860E37
:102B2000E66E010EE66E030EE66E280EE66E74EC9F
:102B300020F0E552E552E552E5520001B39FB39D06
:102B4000B39BB3C0E6FF0F0EE66E59EC20F0E552E2
:102B5000E5520E0EE66EA3EC20F0E552E00B800885
:102B600008E0B3C0E6FF0F0EE66E59EC20F0E55228
:102B7000E552040EE15C02E2E16AE552E16EE552E3
:0A2B8000E7CFD9FF12001200120087
:062B8A0065960F0139877A
:102B9000640EE66EBEEC1FF0E552C4EC1DF00400BE
:102BA000A2EC11F0E7EC11F004000001616B040EDF
:102BB000626F636B0001656B0001646B0001666B03
:102BC000676B686B0001A00E696F6A6B6B6B00012D
:102BD000A00E6C6F6D6B6E6B0001726B61C073F059
:102BE00062C074F063C075F00001786B0001796B0E
:102BF00000017A6B00017B6B7C6B7D6B00016F6B5E
:102C0000706B716B0001816B0001826B0001976B2F
:102C1000986B996B00019A6B9B6B9C6B0001010E8A
:102C2000836F0001010E846F0001856B0001866BCC
:102C300000019D6B9E6B9F6B0001876B0001886B91
:102C40000001A36BA46BA56B0001896B00018A6B6B
:102C500000018D6B00017E6B7F6B806B0001010EAC
:102C60008E6F00018F6B0001A66BA76BA86B000134
:102C7000A96BAA6BAB6B0001906B0001916B00011B
:102C8000926B0001936B0001946B0001956B000146
:102C9000AC6BAD6BAE6B0001AF6BB06BB16B000199
:102CA000630E966F00018F510BE180AE09D061C0B9
:102CB000A6F062C0A7F063C0A8F00001010E8F6FFC
:102CC00080BE02D000018F6B00018F051BE1A60EB4
:102CD000E96E000EEA6EEE500001615D006EEE508E
:102CE00000016259016EEE5000016359026E140E2C
:102CF000001803E1015001E1025004E180AE02D06E
:102D00000EEF00F0040022EC0AF00400F2A425D03B
:102D1000F294480ED76EE40ED66E0001612B000EC1
:102D20006223000E6323730EE96E000EEA6EEE500E
:102D30000001615D006EEE5000016259016EEE50BF
:102D400000016359026E080E005C000E0158000E6F
:102D5000025803E30001010E786F0001790503E1D9
:102D600007EC20F002D0FDEC1FF000017A5101E0E9
:102D700087D17E0EE96E000EEA6EEE500001615DB5
:102D8000006EEE5000016259016EEE500001635971
:102D9000026ED880010E0054000E0154000E025441
:102DA00005E30001790502E100018E6B00018E51FF
:102DB00006E10001795103E10001010E8E6F00016F
:102DC000790556E17B0EE96E000EEA6EEE500001C9
:102DD000615D006EEE5000016259016EEE5000011F
:102DE0006359026E040E005C000E0158000E02587A
:102DF0003FE300018E0535E10001650517E10001A3
:102E0000656B61C069F062C06AF063C06BF000017D
:102E1000A00E6C6F6D6B6E6B89920001010E726F6C
:102E200061C07BF062C07CF063C07DF0000164058E
:102E300017E10001646B61C06CF062C06DF063C0AB
:102E40006EF00001A00E696F6A6B6B6B89900001D8
:102E5000010E726F61C07BF062C07CF063C07DF0D8
:102E600007D000018E0504E10001646B0001656B71
:102E70006C0EE96E000EEA6EEE500001615D006EB0
:102E8000EE5000016259016EEE5000016359026E6E
:102E9000A40E005C000E0158000E025801E2F0D0B2
:102EA000690EE96E000EEA6EEE500001615D006E83
:102EB000EE5000016259016EEE5000016359026E3E
:102EC000A40E005C000E0158000E025801E2D8D09A
:102ED0000001905102E0000E01D0010E036E660E5B
:102EE000E96E000EEA6EEE500001615D006EEE507C
:102EF00000016259016EEE5000016359026E180E16
:102F0000005C000E0158000E025802E3000E01D0D2
:102F1000010E031044E00001655103E10001010EC0
:102F2000926F000192053AE1000165050CE1000194
:102F300090290001906F0001926B61C066F062C041
:102F400067F063C068F0030E0001905D1FE161C08F
:102F500069F062C06AF063C06BF00001A00E6C6F94
:102F60006D6B6E6B89920001656B61C066F062C02B
:102F700067F063C068F00001906B0001010E726F92
:102F800061C07BF062C07CF063C07DF0000164052D
:102F900005E10001010E926F0001906B05D0000168
:102FA000010E926F0001906B0001915102E0000E42
:102FB00001D0010E036E660EE96E000EEA6EEE5051
:102FC0000001615D006EEE5000016259016EEE502D
:102FD00000016359026E180E005C000E0158000ECD
:102FE000025802E3000E01D0010E031044E000017C
:102FF000645103E10001010E936F000193053AE172
:10300000000164050CE1000191290001916F0001AC
:10301000936B61C066F062C067F063C068F0030E36
:103020000001915D1FE161C06CF062C06DF063C092
:103030006EF00001A00E696F6A6B6B6B89900001E6
:10304000646B61C066F062C067F063C068F0000145
:10305000916B0001010E726F61C07BF062C07CF069
:1030600063C07DF00001650505E10001010E936F6D
:103070000001916B05D00001010E936F0001916B6F
:1030800081A2A0D16C0EE96E000EEA6EEE50000136
:10309000615D006EEE5000016259016EEE5000015C
:1030A0006359026EA40E005C000E0158000E025817
:1030B00001E287D1690EE96E000EEA6EEE50000162
:1030C000615D006EEE5000016259016EEE5000012C
:1030D0006359026EA40E005C000E0158000E0258E7
:1030E00001E26FD1AC0EE96E000EEA6EEE50000107
:1030F000615D006EEE5000016259016EEE500001FC
:103100006359026ED880040E0054000E0154000E64
:10311000025401E356D181A404D00001010E8B6F4B
:1031200002D000018B6B81A604D00001010E8C6FD0
:1031300002D000018C6B000187510CE100018B5122
:1031400009E161C0A0F062C0A1F063C0A2F000017B
:10315000010E876F000188510CE100018C5109E1DB
:1031600061C0A3F062C0A4F063C0A5F00001010E2D
:10317000886FA00EE96E000EEA6EEE500001615DF0
:10318000006EEE5000016259016EEE50000163596D
:10319000026E010E001803E1015001E1025009E145
:1031A00000018B5104E10001010E896F02D0000182
:1031B000876BA30EE96E000EEA6EEE500001615DB2
:1031C000006EEE5000016259016EEE50000163592D
:1031D000026E010E001803E1015001E1025009E105
:1031E00000018C5104E10001010E8A6F02D0000140
:1031F000886B6C0EE96E000EEA6EEE500001615DA8
:10320000006EEE5000016259016EEE5000016359EC
:10321000026EA40E005C000E0158000E025801E27E
:103220009AD0690EE96E000EEA6EEE500001615D03
:10323000006EEE5000016259016EEE5000016359BC
:10324000026EA40E005C000E0158000E025801E24E
:1032500082D00001725101E07ED07B0EE96E000E3B
:10326000EA6EEE500001615D006EEE5000016259A1
:10327000016EEE5000016359026ED880080E0054B2
:10328000000E0154000E025466E20001890530E18F
:10329000A00EE96E000EEA6EEE500001615D006E58
:1032A000EE5000016259016EEE5000016359026E4A
:1032B000020E005C000E0158000E025819E30001D6
:1032C0008B0516E10001896B0001876B61C069F015
:1032D00062C06AF063C06BF00001A00E6C6F6D6B92
:1032E0006E6B89920001010E726F0001010E946FE6
:1032F00000018A0530E1A30EE96E000EEA6EEE5081
:103300000001615D006EEE5000016259016EEE50E9
:1033100000016359026E020E005C000E0158000E9F
:10332000025819E300018C0516E100018A6B0001C7
:10333000886B61C06CF062C06DF063C06EF000011C
:10334000A00E696F6A6B6B6B89900001010E726F42
:103350000001010E946FA00EE96E000EEA6EEE50B1
:103360000001615D006EEE5000016259016EEE5089
:1033700000016359026E400E005C000E0158000E01
:10338000025804E30001896B0001876BA30EE96E0C
:10339000000EEA6EEE500001615D006EEE5000011D
:1033A0006259016EEE5000016359026E400E005CDE
:1033B000000E0158000E025804E300018A6B000160
:1033C000886B0FD000018D510CE081B40AD061C030
:1033D00097F062C098F063C099F00001816B000122
:1033E0008D6B81B42ED081B62CD08992899000014A
:1033F000726B0001A40E6C6F6D6B6E6B0001A40EFE
:10340000696F6A6B6B6B61C07BF062C07CF063C0FC
:103410007DF00001876B0001896B0001A06BA16B3F
:10342000A26B0001886B00018A6B0001A36BA46B87
:10343000A56B0001946B61C0ACF062C0ADF063C0DD
:10344000AEF06C0EE96E000EEA6EEE500001615DAA
:10345000006EEE5000016259016EEE50000163599A
:10346000026EA40E005C000E0158000E025865E3C7
:10347000690EE96E000EEA6EEE500001615D006EAD
:10348000EE5000016259016EEE5000016359026E68
:10349000A40E005C000E0158000E02584EE300011D
:1034A000835103E10001010E856F0001830512E1E4
:1034B000000185050FE10001812B0001010E836FE2
:1034C0000001856B0001826B61C09DF062C09EF0BF
:1034D00063C09FF0030E0001815D08E361C097F0B7
:1034E00062C098F063C099F00001816B00018451C3
:1034F00003E10001010E866F0001840512E1000165
:1035000086050FE10001822B0001010E846F00018E
:10351000866B0001816B61C09DF062C09EF063C04C
:103520009FF0030E0001825D08E361C09AF062C063
:103530009BF063C09CF00001826B690EE96E000E87
:10354000EA6EEE500001611908E1EE5000016219C7
:1035500004E1EE500001631900E10DE100018D511D
:103560000AE061C097F062C098F063C099F0000172
:10357000816B00018D6B00018151000182250008E3
:1035800026E29D0EE96E000EEA6EEE500001615DCE
:10359000006EEE5000016259016EEE500001635959
:1035A000026ED8800C0E0054000E0154000E02541E
:1035B0000EE20001816B0001826B0001010E836F3E
:1035C0000001856B0001010E846F0001866B970E70
:1035D000E96E000EEA6EEE500001615D006EEE5085
:1035E00000016259016EEE5000016359026ED880ED
:1035F000140E0054000E0154000E025405E36AEC50
:1036000022F000018D6B02D060EC22F09A0EE96E80
:10361000000EEA6EEE500001615D006EEE5000019A
:103620006259016EEE5000016359026ED880140E8B
:103630000054000E0154000E025406E37EEC22F00A
:103640000001010E8D6F02D074EC22F0970EE96E2E
:10365000000EEA6EEE500001615D006EEE5000015A
:103660006259016EEE5000016359026ED880140E4B
:103670000054000E0154000E025418E30001815161
:1036800000018225000812E20001976B986B996B8C
:103690000001816B0001826B0001010E836F00014C
:1036A000856B0001010E846F0001866B9A0EE96E36
:1036B000000EEA6EEE500001615D006EEE500001FA
:1036C0006259016EEE5000016359026ED880140EEB
:1036D0000054000E0154000E025418E30001815101
:1036E00000018225000812E200019A6B9B6B9C6B23
:1036F0000001816B0001826B0001010E836F0001EC
:10370000856B0001010E846F0001866B6F0EE96E00
:10371000000EEA6EEE500001615D006EEE50000199
:103720006259016EEE5000016359026ED880080E96
:103730000054000E0154000E025402E3899235D069
:103740006C0EE96E000EEA6EEE500001615D006ED7
:10375000EE5000016259016EEE5000016359026E95
:10376000A00E005C000E0158000E02581EE26C0E06
:10377000E96E000EEA6EEE500001615D006EEE50E3
:1037800000016259016EEE5000016359026E020E93
:10379000001803E1015001E1025007E00001720549
:1037A00004E10001940501E189826F0EE96E000ECB
:1037B000EA6EEE500001615D006EEE50000162594C
:1037C000016EEE5000016359026ED880080E00545D
:1037D000000E0154000E025402E3899035D0690EA8
:1037E000E96E000EEA6EEE500001615D006EEE5073
:1037F00000016259016EEE5000016359026EA00E85
:10380000005C000E0158000E02581EE2690EE96EBF
:10381000000EEA6EEE500001615D006EEE50000198
:103820006259016EEE5000016359026E020E0018DB
:1038300003E1015001E1025007E00001720504E1DB
:103840000001940501E189806C0EE96E000EEA6EBC
:10385000EE500001615D006EEE5000016259016E94
:10386000EE5000016359026EA00E005C000E01587C
:10387000000E02581DE3690EE96E000EEA6EEE506E
:103880000001615D006EEE5000016259016EEE5064
:1038900000016359026EA00E005C000E0158000E7C
:1038A000025806E3899289900001726B0001946BC3
:1038B0006C0EE96E000EEA6EEE500001615D006E66
:1038C000EE5000016259016EEE5000016359026E24
:1038D000020E001803E1015001E1025004E1000171
:1038E000965101E18992690EE96E000EEA6EEE5082
:1038F0000001615D006EEE5000016259016EEE50F4
:1039000000016359026E020E001803E1015001E14B
:10391000025004E10001960501E189906C0EE96E08
:10392000000EEA6EEE500001615D006EEE50000187
:103930006259016EEE5000016359026E280E0018A4
:1039400003E1015001E102501FE1000196511CE129
:10395000899289900001726B0001A40E6C6F6D6BEF
:103960006E6B0001A40E696F6A6B6B6B61C07BF0BC
:1039700062C07CF063C07DF00001946B61C0ACF06C
:1039800062C0ADF063C0AEF0690EE96E000EEA6E83
:10399000EE500001615D006EEE5000016259016E53
:1039A000EE5000016359026E110E001803E1015040
:1039B00001E102501FE1000196051CE18992899006
:1039C0000001726B0001A40E6C6F6D6B6E6B0001D9
:1039D000A40E696F6A6B6B6B61C07BF062C07CF098
:1039E00063C07DF00001946B61C0ACF062C0ADF0CB
:1039F00063C0AEF0730EE96E000EEA6EEE50000189
:103A0000615D006EEE5000016259016EEE500001E2
:103A10006359026ED880F00E0054000E0154000E5F
:103A2000025401E3AED0898A010EE66E010EE66E05
:103A30002B0EE66E22EC22F0E552E552E552F19CA7
:103A4000F292F28804000300F2A282D00400000186
:103A5000010E956F010EE66EBEEC1FF0E552E66AB0
:103A6000010EE66E2B0EE66E22EC22F0E552E552D8
:103A7000E552E66A010EE66E2C0EE66E22EC22F0AE
:103A8000E552E552E552F298F292899A0001B39F0D
:103A90000001B39D0001B39BB3C0E6FF0F0EE66EBD
:103AA00059EC20F0E552E5520E0EE66EA3EC20F044
:103AB000E552E00B08E0B3C0E6FF0F0EE66E59ECEE
:103AC00020F0E552E5520001616B040E626F636BFA
:103AD0000001666B676B686B0001A00E696F6A6B13
:103AE0006B6B0001A00E6C6F6D6B6E6B00017B6BDE
:103AF0007C6B7D6B00016F6B706B716B0001976B62
:103B0000986B996B00019A6B9B6B9C6B00019D6B92
:103B10009E6B9F6B0001A36BA46BA56B00017E6B7A
:103B20007F6B806B0001A66BA76BA86B0001A96B74
:103B3000AA6BAB6B0001AC6BAD6BAE6B0001AF6BF6
:103B4000B06BB16B61C073F062C074F063C075F0AC
:103B500007EC20F0050EE66E25EC20F0E552FDECBA
:103B60001FF080AE07D061C073F062C074F063C014
:103B700075F007D00001950503E10001956B01D0B8
:103B800062D752EF16F012000F011F0E486F0F019F
:103B90001F0E496F9B8CFC0ED3140009D36E9482C8
:103BA000949C8B9C94948B940E01550EA76EAA0E38
:103BB000A76EFF910C0EFB6F0A0ED76F090ED36F25
:103BC000550EA76EAA0EA76EFF81929089909292D1
:103BD00089929294898492968986929A899A929CE3
:103BE000898C928E9382F19E94908B80938493869D
:083BF000938A949EC08012002C
:083BF8008994C00EE66E4BEC4F
:103C000023F0E55289840001DA6BDA51006E016A13
:103C1000D890015004E6FF0E005C000E015802E24D
:103C2000DA2BF3D71200D9CFE6FFE1CFD9FF899481
:103C3000020EE66E4BEC23F0E552FE0EDBCFE6FF04
:103C40004BEC23F0E552FD0EDBCFE6FF4BEC23F00F
:103C5000E5528984E552E7CFD9FF1200D9CFE6FFBC
:103C6000E1CFD9FFE6528994020EE66E4BEC23F0C9
:103C7000E552FE0EDBCFE6FF4BEC23F0E552DF6AA8
:103C8000FD0EDB50DF5C13E2DF50E76EFB0EDBCF97
:103C9000E9FFFC0EDBCFEAFFE750E926000EEA223F
:103CA000EF50E66E4BEC23F0E552DF2AE9D789842A
:103CB000E552E552E7CFD9FF1200D9CFE6FFE1CFB9
:103CC000D9FFE6528994030EE66E4BEC23F0E552E1
:103CD000FE0EDBCFE6FF4BEC23F0E55280EC23F049
:103CE000DF6E8984DF50E552E552E7CFD9FF12003D
:103CF000D9CFE6FFE1CFD9FFE6528994030EE66EF5
:103D00004BEC23F0E552FE0EDBCFE6FF4BEC23F04D
:103D1000E552DF6AFD0EDB50DF5C14E280EC23F03D
:103D2000E66EDF50E76EFB0EDBCFE9FFFC0EDBCF6C
:103D3000EAFFE750E926000EEA22E552E750EF6E6F
:103D4000DF2AE8D780EC23F0E66EDF50E76EFB0E4B
:103D5000DBCFE9FFFC0EDBCFEAFFE750E926000EE0
:103D6000EA22E552E750EF6E8984E552E552E7CF4B
:103D7000D9FF1200D9CFE6FFE1CFD9FFE6528994EF
:103D8000FE0EDBCFE6FF4BEC23F0E552DF6AFD0EC3
:103D9000DB50DF5C14E280EC23F0E66EDF50E76E70
:103DA000FB0EDBCFE9FFFC0EDBCFEAFFE750E92695
:103DB000000EEA22E552E750EF6EDF2AE8D780ECEA
:103DC00023F0E66EDF50E76EFB0EDBCFE9FFFC0E63
:103DD000DBCFEAFFE750E926000EEA22E552E75082
:103DE000EF6E8984E552E552E7CFD9FF1200D9CFB3
:103DF000E6FFE1CFD9FF030EE126FE0EDB50FF0800
:103E000038E1A7D8DF6EDFBC07D0440EF36EFE0E9C
:103E1000F3CFDBFF840E29D0DFB807D0420EF36E5C
:103E2000FE0EF3CFDBFF820E20D0DFA418D0540E9D
:103E3000DF141FE0E66A300EE66EF5DEE552E5526D
:103E40000001DA6BDA51006E016AD890015004E685
:103E5000FF0E005C000E015802E2DA2BF3D7400E91
:103E6000F36EFE0EF3CFDBFF810EF36E020EF3CF87
:103E7000DBFF8994FE0EDBCFE6FF4BEC23F0E5522F
:103E8000DF6AFD0EDB50DF5C13E2DF50E76EFB0EF6
:103E9000DBCFE9FFFC0EDBCFEAFFE750E926000E9F
:103EA000EA22EF50E66E4BEC23F0E552DF2AE9D729
:103EB0008984020EDBCFE6FF0FD8E552FE0EDB5001
:103EC000006E030EE15C02E2E16AE552E16E005031
:103ED000E552E7CFD9FF1200D9CFE6FFE1CFD9FFF6
:103EE000E652FE0EDBA00ED0E66A300EE66E9BDEDA
:103EF000E552E5528994FE0EDBCFE6FF4BEC23F052
:103F0000E5528984FE0EDBA20ED0E66A400EE66E14
:103F10008ADEE552E5528994FE0EDBCFE6FF4BECDC
:103F200023F0E5528984FE0EDBA40ED0E66A500E23
:103F3000E66E79DEE552E5528994FE0EDBCFE6FFB0
:103F40004BEC23F0E5528984E552E552E7CFD9FFE7
:103F50001200D9CFE6FFE1CFD9FFE6528994A00E37
:103F6000E66E4BEC23F0E55280EC23F0DF6E8984A3
:103F7000DF50E552E552E7CFD9FF1200D9CFE6FF77
:103F8000E1CFD9FFE652CF0ECF6E2B0ECE6ECD8095
:103F9000DF6AFE0EDB50DF5C09E29EA0FED79E903A
:103FA000CF0ECF6E2B0ECE6EDF2AF3D7CD90E5521B
:103FB000E552E7CFD9FF1200D9CFE6FFE1CFD9FF15
:103FC0008994050EE66E4BEC23F0E552FE0EDBCF36
:103FD000E6FF4BEC23F0E552FD0EDBCFE6FF4BECAA
:103FE00023F0E552FC0EDBCFE6FF4BEC23F0E5526D
:103FF0008984E552E7CFD9FF1200E668100EE66E1D
:104000000C0EE66ED9DFE552E552E5521200E66A83
:10401000100EE66E0C0EE66ECFDFE552E552E5526D
:104020001200E668200EE66E0C0EE66EC5DFE55265
:10403000E552E5521200E66A200EE66E0C0EE66EC0
:10404000BBDFE552E552E5521200D9CFE6FFE1CFE2
:10405000D9FFE652350ECF6ECE6ACD80DF6AFE0EF6
:10406000DB50DF5C09E29EA0FED79E90CF0ECF6EA4
:104070002B0ECE6EDF2AF3D7CD90E552E552E7CF77
:04408000D9FF120052
:0C4084008996C00EE66E2DEC23F0E5528C
:1040900089860001DB6BDB51006E016AD89001500C
:1040A00004E6FF0E005C000E015802E2DB2BF3D7A2
:1040B0001200D9CFE6FFE1CFD9FF8996020EE66E56
:1040C0002DEC23F0E552FE0EDBCFE6FF2DEC23F0C6
:1040D000E552FD0EDBCFE6FF2DEC23F0E55289869D
:1040E000E552E7CFD9FF1200D9CFE6FFE1CFD9FFE4
:1040F000E6528996020EE66E2DEC23F0E552FE0E96
:10410000DBCFE6FF2DEC23F0E552DF6AFD0EDB503E
:10411000DF5C13E2DF50E76EFB0EDBCFE9FFFC0E46
:10412000DBCFEAFFE750E926000EEA22EF50E66E09
:104130002DEC23F0E552DF2AE9D78986E552E552D6
:10414000E7CFD9FF1200D9CFE6FFE1CFD9FFE65282
:104150008996030EE66E2DEC23F0E552FE0EDBCFC2
:10416000E6FF2DEC23F0E55269EC23F0DF6E898643
:10417000DF50E552E552E7CFD9FF1200D9CFE6FF75
:10418000E1CFD9FFE6528996030EE66E2DEC23F0BF
:10419000E552FE0EDBCFE6FF2DEC23F0E552DF6AA1
:1041A000FD0EDB50DF5C14E269EC23F0E66EDF50BD
:1041B000E76EFB0EDBCFE9FFFC0EDBCFEAFFE7503B
:1041C000E926000EEA22E552E750EF6EDF2AE8D733
:1041D00069EC23F0E66EDF50E76EFB0EDBCFE9FF04
:1041E000FC0EDBCFEAFFE750E926000EEA22E5529B
:1041F000E750EF6E8986E552E552E7CFD9FF12000E
:10420000D9CFE6FFE1CFD9FFE6528996FE0EDBCF8C
:10421000E6FF2DEC23F0E552DF6AFD0EDB50DF5C9C
:1042200014E269EC23F0E66EDF50E76EFB0EDBCFA5
:10423000E9FFFC0EDBCFEAFFE750E926000EEA2299
:10424000E552E750EF6EDF2AE8D769EC23F0E66E1F
:10425000DF50E76EFB0EDBCFE9FFFC0EDBCFEAFFA2
:10426000E750E926000EEA22E552E750EF6E898614
:10427000E552E552E7CFD9FF1200D9CFE6FFE1CFF3
:10428000D9FF030EE126FE0EDB50FF0838E1A7D868
:10429000DF6EDFBC07D0440EF36EFE0EF3CFDBFF04
:1042A000840E29D0DFB807D0420EF36EFE0EF3CF96
:1042B000DBFF820E20D0DFA418D0540EDF141FE0E5
:1042C000E66A300EE66EF5DEE552E5520001DB6B84
:1042D000DB51006E016AD890015004E6FF0E005CCD
:1042E000000E015802E2DB2BF3D7400EF36EFE0EF8
:1042F000F3CFDBFF810EF36E020EF3CFDBFF899667
:10430000FE0EDBCFE6FF2DEC23F0E552DF6AFD0E5B
:10431000DB50DF5C13E2DF50E76EFB0EDBCFE9FF23
:10432000FC0EDBCFEAFFE750E926000EEA22EF5051
:10433000E66E2DEC23F0E552DF2AE9D78986020EDE
:10434000DBCFE6FF0FD8E552FE0EDB50006E030E0A
:10435000E15C02E2E16AE552E16E0050E552E7CF2E
:10436000D9FF1200D9CFE6FFE1CFD9FFE652FE0E0A
:10437000DBA00ED0E66A300EE66E9BDEE552E5521B
:104380008996FE0EDBCFE6FF2DEC23F0E552898601
:10439000FE0EDBA20ED0E66A400EE66E8ADEE55225
:1043A000E5528996FE0EDBCFE6FF2DEC23F0E552B9
:1043B0008986FE0EDBA40ED0E66A500EE66E79DE2C
:1043C000E552E5528996FE0EDBCFE6FF2DEC23F099
:1043D000E5528986E552E552E7CFD9FF1200D9CFE1
:1043E000E6FFE1CFD9FFE6528996A00EE66E2DECEE
:1043F00023F0E55269EC23F0DF6E8986DF50E55249
:10440000E552E7CFD9FF1200D9CFE6FFE1CFD9FFC0
:10441000E652CF0ECF6E2B0ECE6ECD80DF6AFE0E33
:10442000DB50DF5C09E29EA0FED79E90CF0ECF6EE0
:104430002B0ECE6EDF2AF3D7CD90E552E552E7CFB3
:10444000D9FF1200D9CFE6FFE1CFD9FF8996050E3B
:10445000E66E2DEC23F0E552FE0EDBCFE6FF2DECF1
:1044600023F0E552FD0EDBCFE6FF2DEC23F0E55205
:10447000FC0EDBCFE6FF2DEC23F0E5528986E552FA
:10448000E7CFD9FF1200D9CFE6FFE1CFD9FFE6523F
:10449000350ECF6ECE6ACD80DF6AFE0EDB50DF5C5C
:1044A00009E29EA0FED79E90CF0ECF6E2B0ECE6E51
:1044B000DF2AF3D7CD90E552E552E7CFD9FF1200BE
:1044C000E66A100EE66E0C0EE66EBCDFE552E552B3
:1044D000E5521200E668100EE66E0C0EE66EB2DFD4
:1044E000E552E552E5521200E66A200EE66E0C0E29
:1044F000E66EA8DFE552E552E5521200E668200EAE
:10450000E66E0C0EE66E9EDFE552E552E5521200B5
:104510002A0EF66E140EF76E000EF86E00010900FA
:10452000F550D16F0900F550D26F03E1D16701D08A
:104530003DD00900F550CC6F0900F550CD6F090052
:10454000F550CE6F09000900F550E96E0900F550ED
:10455000EA6E090009000900F550CF6F0900F55017
:10456000D06F09000900F6CFD3F0F7CFD4F0F8CF21
:10457000D5F0CCC0F6FFCDC0F7FFCEC0F8FF0001EC
:10458000CF5302E1D05307E00900F550EE6ECF079C
:10459000F8E2D007F9D7D3C0F6FFD4C0F7FFD5C0F3
:0E45A000F8FF0001D107000ED25BBFD712005A
:0245AE00D9CF63
:1045B000E6FFDACFE6FFE1CFD9FFE2CFDAFF3F0E29
:1045C0007316726AFD0EDB507212FB0EDB50731213
:1045D000FC0EDB50030A09E0010A04E0020A06E1CE
:1045E000738C04D0738C728801D07288FD0EDB50FE
:1045F000050A01E0010A728AE552E5CFDAFFE7CF4A
:04460000D9FF1200CC
:0C460400D9CFE6FFDACFE6FFE1CFD9FF07
:10461000E2CFDAFF3F0EC716C66AFD0EDB50C612A8
:10462000FB0EDB50C712FC0EDB50030A09E0010A47
:1046300004E0020A06E1C78C04D0C78CC68801D00A
:10464000C688FD0EDB50050A01E0010AC68AE55264
:0A465000E5CFDAFFE7CFD9FF120033
:06465A00D9CFE6FFDACF24
:10466000E6FFE1CFD9FFE2CFDAFFE6527550DF6E09
:10467000A49E729EFD0EDB50756E72AE02D0FF0ED0
:1046800003D0A4AEFED7000EE552E552E5CFDAFF27
:06469000E7CFD9FF120084
:0A469600D9CFE6FFDACFE6FFE1CF4F
:1046A000D9FFE2CFDAFFE652C950DF6E9E96C69E72
:1046B000FD0EDB50C96EC6AE02D0FF0E03D09EA623
:1046C000FED7000EE552E552E5CFDAFFE7CFD9FF7E
:0246D0001200D6
:0E46D200D9CFE6FFDACFE6FFE1CFD9FFE2CF86
:1046E000DAFFE6527550DF6EA49E756AA4AEFED75F
:1046F0007550E552E552E5CFDAFFE7CFD9FF12005A
:10470000D9CFE6FFDACFE6FFE1CFD9FFE2CFDAFF7C
:10471000E652C950DF6E9E96C96A9EA6FED7C95062
:0E472000E552E552E5CFDAFFE7CFD9FF1200F0
:02472E00C00EBB
:10473000F36E00EE00F00E0E01D81200EA6002D017
:0E474000EE6AFCD7F350E9601200EE6AFCD777
:02474E001DEE5E
:1047500000F02DEE00F0F86A069C88EC22F0B5EC33
:0A47600023F0C5EC15F0FBD71200A2
:02476A0012003B
:04476C000000000049
:0B4770000001F00000000080000100CC
:017FF8008CFC
:017FF900F790
:017FFA000284
:017FFB00F88D
:017FFC00F193
:017FFD00F88B
:017FFE00DFA3
:017FFF00F190
:00000001FF
